:08000000F0FF0220513C00005A
:100400000000000000000001FFFFFFFFBE03FFFF30
:1004100008B5164804F07EFD154804F07BFD15482C
:1004200004F078FD144804F075FD0C214FF40040F1
:1004300004F076FD114804F06DFD0C21104804F025
:100440006FFD104804F066FD0F4804F063FD0F488F
:1004500004F060FD0E4804F05DFD0E4804F05AFD06
:100460000D48BDE8084004F055BD00BF156200000E
:1004700030620000356200005662000058620000E1
:10048000FF7F02005A6200005E620000706200009E
:100490008362000096620000A8620000A0F13003B1
:1004A0000246D8B2092807D9A2F13703D8B20F28DB
:1004B00084BFA2F15700C0B27047000010B592B0DF
:1004C0002022002104460AA805F07AFD11221749CE
:1004D00009920AA804F006FC12AA002152F8243D51
:1004E00058201F2B1DD901B10993002C14BF4FF4C4
:1004F000A0504FF4C0500AA94FF4807203F086FC5C
:100500000E220B4901A804F0EDFB45F6580300222A
:1005100001A94FF40050ADF8123003F077FC12B08F
:1005200010BD0133D118C8700121DAE75460000012
:10053000C36200002DE9F04F0378A3B003F0DF039E
:100540000024532B064604918DF8214040F0AE80E4
:10055000DDE906A19DF820700294A346A14603940C
:100560000194A04622469CE00A2A02F101052ADCF9
:10057000042A307880F2A680022A00F39980012AAA
:1005800080F28580002A56D0022398FBF3F222AB3A
:100590001A4418F0010F3078059200F0EE80FFF752
:1005A0007DFF059A019B12F866CC40EA0C00C0B2B0
:1005B00002F8660C1844C3B2019308F1010888459B
:1005C000A8BFC8256CE0C82ADEDBC92A40F39180A9
:1005D000CA2AD9D1039B0BB1CDF818A0029B0BB14D
:1005E0008DF82190BBF1000F00D007910CB18DF870
:1005F0002070069A0199130C03EB1263134403EB6A
:1006000012231944CB439DF8211003F0FF039942B4
:1006100040F0C580022398FBF3F8B8F1000F45DDE8
:1006200048F207039A4200F2A580B2F5004F80F02D
:100630009C80052005E03028074601D0352803D1ED
:10064000002023B0BDE8F08FA0F13704022C00F2A7
:100650009B80039B0BB1CDF818A0029B0BB18DF8CA
:100660002190BBF1000F00D00791002211468DF8B8
:100670002000104603F08AF808224A494FF400404F
:1006800003F084F8002800F088800120D9E7FFF704
:1006900005FFC5F103039B00984001434FF0010B98
:1006A0002A46049B01369E42FFF45EAF0220C8E753
:1006B000CBB2312F01934FEA41010ED106394FF0F1
:1006C000010B0825FFF7EAFEC5F10B0292009040EE
:1006D00001234AEA000A0393E2E7322F03BF0839F5
:1006E0004FF0010B06250A391CBF4FF0010B042502
:1006F000E8E73078FFF7D2FEC5F1CA0292009040D9
:1007000040EA090901235FFA89F90293C8E7C11891
:10071000A1F5004115F8014B0C700133B8F1010847
:1007200006938DD0069B9342F1D9069B03EB0802FA
:10073000B2F5203F3FF67DAF1B4C226852B1934289
:1007400008D0534033F0070304D00022114610466E
:1007500003F01CF842462946069803F017F80028D3
:1007600093D1069B434423606BE70DF122051A46A3
:100770000C48D7E70DF12205D7E7FFF78FFE059A62
:10078000000102F8660C18E701241146A346029402
:10079000914603949246254682E7072051E70420BC
:1007A0004FE700BFA802FF1FB803FF1F0A448A4299
:1007B00000D1704740BA11F8013B80B24340C3F307
:1007C0000310584080EA003000B2430103F4FF53A5
:1007D000584080B2EBE7000008B54FF400431B68B7
:1007E000013340D048F204031B6801333BD000289A
:1007F00033D002F08FFA1C4B1C4900221A600B68A0
:1008000023F4872323F480630B6051F80C3C23F41A
:10081000406341F80C3C164B1A60164A136823F4E7
:10082000003323F006031360A2F581520C3A1368DB
:1008300043F08073136052F8043C23F0004342F805
:10084000043C0D4A4FF0FF33136053609360C2F8CD
:100850000031C2F80431C2F808314FF40040BDE85D
:10086000084003F0CDBA08BD10E000E03480044039
:10087000800590423080044080E100E02DE9F8439B
:10088000954C867B23683BB9944B954A1B78137033
:10089000944A137001232360934D01270522924946
:1008A000304604F0BFF870B9904E914DB0462968BB
:1008B000DFF82C920122314499F8000004F0B2F8DC
:1008C00078B9BDE8F883EB78002BE7D12B79012BC1
:1008D00002D103F081F9E1E70120FFF77DFF2760F6
:1008E000DCE72F68F35D0A2BE1D02268042A00F0D0
:1008F000B78012DC012A1DD0022A15D198F80030E9
:1009000003F0DF03592B40F0A980202A40F09080AB
:10091000784804F0FFFA40232CE0202AEED0402A49
:10092000ECD0102A00F0D2802B68FF2BC4BF00232C
:100930002B60BCE70D2B62D10023022F2B605CD112
:10094000337803F0DF03442B09D1737803F0DF031E
:10095000432B52D1684804F0DDFA2760E4E74C2BC2
:100960000AD1737803F0DF03442B46D1634804F0C7
:10097000D1FA04232360D7E7472B0FD198F8013031
:1009800003F0DF034F2B38D15D4804F0C3FA022295
:100990000421612004F08CFC0823EBE74D2B0AD1E5
:1009A00098F8013003F0DF03452B26D1554804F0B9
:1009B000B1FA2023DEE7422B1FD198F8013003F073
:1009C000DF03432B19D1504804F0A4FA4FF4004040
:1009D0000378FF2B07D10130B0F5203FF8D14B4809
:1009E00004F098FAA0E7B0F5203FF8D20028F6D03E
:1009F0002C2104F095FA4648F2E74648F0E73F2BF1
:100A000004D100232B60FFF703FD8DE7F11999F85E
:100A1000000004F04BFA2B68F15C5A1C08292A608C
:100A200082D1012A02DC00232B607DE7013BFBE73A
:100A3000402A02D102F074FE76E7374804F06AFAE1
:100A40004FF400314FF4004002F070FE20B93348FB
:100A500004F060FA01238DE73148F9E73148F7E700
:100A6000032B07D1304804F055FA00232B60FFF721
:100A7000CFFCEFE7791C0D2B29607FF455AF314493
:100A80004046FFF757FD013806281DD8DFE800F083
:100A90000C041C0A181C0E00244804F03BFA102316
:100AA0002360C0E72248F8E72248F6E7224804F02E
:100AB00031FA01221421612004F0FAFB0823EFE748
:100AC0001E4804F027FAAEE71D48FAE7122B7FF420
:100AD0002BAF01225CE700BFA002FF1FBC03FF1F7A
:100AE0009C02FF1F9802FF1FB002FF1FB502FF1FED
:100AF000A402FF1F09610000666000007F60000023
:100B00009F600000B9600000D1600000E560000057
:100B1000F1600000016100003C61000050610000D4
:100B20005F6100006C6100007C6100008861000072
:100B3000AC610000CC610000F561000013620000B0
:100B40004E610000064B1B6813F0020F10B5054CF8
:100B500003D000202080FFF73FFE0023238010BD3C
:100B600090F00F40FEFF0220F8B506460D461446F1
:100B70001AB1022A47D0002418E0027822F080033C
:100B8000212B38D1C179837943EA01231F49120609
:100B90000B8043782BD5212B2DD10A21752004F011
:100BA000C9F9082D21D9083DADB20836174F38884C
:100BB000D8B1174C2278202A0BD1072828BF07204C
:100BC000144B85422A46314628BF0246181A04F0C3
:100BD00089F83B88AB424FF0000288BF5D1B227052
:100BE00099BF3A8003243D8006242046F8BD202B7F
:100BF00003D0222B05D00424F7E7054A06241370FE
:100C0000CFE70324CDE70024EFE700BFC603FF1FB3
:100C1000C503FF1FC503FF1F2DE9F0413B4D867B38
:100C20002C78A0B094BB0123ADF80A30384B8DF876
:100C30000E40CDE9003440F20133ADF810306A4681
:100C40007523214605208DF8123003F069FF6123DA
:100C50008DF812302F4B28704FF00122CDE901237F
:100C600021462D4B03936A460520009403F058FF5C
:100C70002A4B8DF8124018706A460323214605203E
:100C8000ADF80E30CDE9004403F04AFF244C254F67
:100C9000DFF89C8005226946304603F0C3FE10B998
:100CA00020B0BDE8F0819DF8030001280ED0752822
:100CB000F0D19DF804200DF10501304603F0B2FE9D
:100CC0009DF80530FE2BE5D1174811E09DF8043062
:100CD000CA2B15D007D80A2BDCD107221349287854
:100CE00004F0E4F8D6E7CB2B05D0CC2BD2D140468C
:100CF00004F010F9CEE7002104F058FE3846F7E77B
:100D00000021022004F052FE2046F1E7BD03FF1F40
:100D1000690B00008000100040000201BC03FF1FAF
:100D2000556300004563000062630000BE03FF1FBF
:100D300039630000122303800048704727630000D6
:100D40004B23038000487047D262000005289FBFF4
:100D5000034B53F8200003780B8088BF00207047B6
:100D60009C63000038B504460D4611F9012B32B9D9
:100D700094F90000003018BF0120404238BD2A2AF3
:100D80000BD1013529462046FFF7ECFF0028F5D0AE
:100D900014F9013B002BF5D104E03F2A94F900300F
:100DA00003D163B94FF0FF30E8E7934207D0D0B2E8
:100DB000A0F14105192D04D8203B9A42F2D101340B
:100DC000D2E761381928EDD82033F6E730B1094B66
:100DD0001B689B070DD50120FFF7FEBC064A136870
:100DE0000133022B1360F2DC02221421532004F0A1
:100DF0005FBA704790F00F408004FF1FF0B5831E6C
:100E0000C1B00446052B59D8DFE803F0030E3F6557
:100E100085BE784B00201860774B1880774B4FF4D5
:100E200000421A60FFF74AFB754C734D714E4FF448
:100E300080726946204601F0A5FD228E2888694609
:100E4000FFF7B4FC336828807BB96C4D238E6A466B
:100E500069464FF4007003F03FF8228E2868694617
:100E600004F07BF860B101233360238EB3F5807FFB
:100E700014BF042403240121532004F05BF81DE077
:100E80002B68228E13442B60EFE75B4C5D49208872
:100E90000622FFF78BFC5C4B2080DB88834217D156
:100EA000544B1B686BB14FF400314FF4004002F01B
:100EB0003DFC0121532004F03DF80524204641B0BB
:100EC000F0BD01221E21532004F0F2F90124F5E7C0
:100ED00001221421F7E7494C49484FF4004300220E
:100EE0000821236001F052FE20226946444801F0A7
:100EF00049FD2368002020332360FFF7DFFA6A46AC
:100F0000694620234FF4007002F0E6FF2022694674
:100F10003E4803F0E7FE3A4C384D4FF48072694684
:100F2000204601F02FFD238E6A4669464FF400707B
:100F300002F0D2FF228E2868694602F027FC238E39
:100F40002868B3F5807F184428601BD00022114622
:100F500002F01CFC4FF4004020222C49286002F0D3
:100F600015FC00221146286802F010FC224B0022DA
:100F70001A80A368264A083B012013600724FFF764
:100F80009DFA78E7062476E7214E1C4F33683968CE
:100F9000194DFF2B15D94FF4807318466A4602F09D
:100FA0009BFF4FF4807269462888FFF7FFFB336888
:100FB0002880A3F5807333603B6803F580733B6042
:100FC00059E76A464FF4807002F086FF326828883D
:100FD0006946FFF7EBFB06220A492880FFF7E6FB8C
:100FE000094B2880DB8883423FF46BAF02225021FB
:100FF00069E700BF7C04FF1FB804FF1F8404FF1FC4
:10100000BC04FF1FD16300007004FF1F8C04FF1F8E
:10101000B404FF1F574B2DE9F0471C681D46E4B18F
:1010200090F80E90544FDFF870A1DFF854815249C8
:101030000522484603F0F6FC08B3F8783C7900280E
:101040004BD1022C45D101F00FFD038B0BB1D9051B
:1010500017D50020FFF7BAFEE9E701221A60FF2149
:101060002022464803F035FE02221421532004F0CA
:101070001FF92146204601F023FB414B1860BDE8D3
:10108000F0871A07E5D45326D8F800103D488AF8AF
:10109000376001F02DFB002815DB3B4B3B493948FD
:1010A00001229A813A4A1A6090221A8118221A75EE
:1010B000D8F800300B6001F0C3FC02215320BDE8DA
:1010C000F04703F037BF01221421304604F0F0F856
:1010D000ADE7012CABD12046BCE7022C47D12A4E0C
:1010E0002A48314601F072F90F3039D0737D9B06E2
:1010F000E3D57489B37D2749E31A254C1C44204667
:10110000FFF730FE0028D8D1234E1D4A0123126874
:101110003146204601F0B0FC0228CED1B2681F4B08
:101120009A42CAD81E4C08222146304601F02AFCB9
:10113000E388B1685BBAE380A3885BBA9AB2A38004
:1011400023681BBA236008339942B6D141F2342395
:101150009A42B2D102202860FFF750FE28608EE745
:10116000012214215320BDE8F04704F0A1B82868FB
:10117000F2E700BF7804FF1FAC04FF1F8C04FF1FC1
:101180008804FF1F586200005804FF1FF404FF1F6B
:10119000C803FF1FB8630000BC04FF1F0800020063
:1011A0007004FF1F10B404688C4203460AD0196013
:1011B000064A90F8484052F82440426923465DF8B8
:1011C000044B184700205DF8044B70471405FF1FBF
:1011D00070B51446BDF810209D18B5F5007F056860
:1011E000C4BFC3F5007292B28D420AD090F8485045
:1011F0000492074A52F825502246AC46BDE870409A
:10120000604741692046194403F06CFD002070BD21
:101210001805FF1F7FB54A68836801324A6090F85D
:101220002B600D46D11AB1FBF6F306FB13130446EF
:10123000002B32D1018B4E0431D5C16802318A4274
:101240003CD02AD32968066ACBB2022200925B0006
:101250000DF10A0206EB1121FFF7BAFF18B16FF08A
:10126000030004B070BDBDF80A300393039A6368AD
:10127000934226D2636A9A4223D82A60E16894F89E
:101280002B3003FB0212218B6A60490405D5012B28
:1012900003D9C3F1010313446B600020E1E729681F
:1012A000066A01F07F03042200929B0003AA06EB6A
:1012B000D111FFF78DFF0028D1D1D7E76FF00800DB
:1012C000CFE76FF00600CCE738B50C4B0C4D012290
:1012D0001A600446022208214D2003F0E9FF1CB1E8
:1012E0004FF400732B8338BD064803F013FE4FF410
:1012F00080732B83044B1C60F5E700BF2805FF1F9C
:101300008005FF1FF06300002405FF1F084A0948FD
:1013100008B5138B43F008031383074B32221A607E
:1013200003F0F8FD0548BDE8084003F0F3BD00BF39
:101330008005FF1FD76300002805FF1FE66300003C
:1013400010B50D4C0D4B94F84820216853F822300D
:1013500062692046984750B9636993F8FE21552A7F
:1013600006D193F8FF31AA2B18BF6FF0020010BD11
:101370006FF00200FBE700BF8005FF1F1405FF1F91
:101380002DE9F743204C214E2368174613F0020243
:1013900002D052B9306828E0028B43F002035206B3
:1013A00023601B4B58BF49021960DFF86490194D48
:1013B0004FF01108D9F8003016482B711A0E6A70D8
:1013C0001A0CAA701A0AEA700DF10701002285F8BA
:1013D00000806A7102F07CFA431C3060EAD0002879
:1013E00006DA236823F00203236003B0BDE8F0832C
:1013F0009DF807301BB9384602F06AFB306023685D
:1014000023F002032360C5E72405FF1F2005FF1F0B
:101410004005FF1F2C05FF1F2DE9F743224C164600
:1014200022681F4612F0020302D053B9002027E0C1
:10143000038B58061D4B58BF490242F0020222603E
:101440001960DFF868901A4D4FF01108D9F80020A4
:101450002A71130E6B70130CAB700DF10701130A98
:101460001348EB70002285F800806A7102F030FAB0
:10147000431CEBD0002806DA236823F00203236024
:1014800003B0BDE8F0839DF807303BB9BDF82820D4
:101490003A4492B23946304602F05AFB236823F0B0
:1014A00002032360C2E700BF2405FF1F3C05FF1FA6
:1014B0002C05FF1F2DE9F04F8FB002F40043069377
:1014C000C2F3C033079391F83A300493D0E9006730
:1014D0008A46B04B0499542201FB023304460C2285
:1014E00039460BA8089303F0FDFB96F900305C2BFE
:1014F00001D02F2B00D101364FF0000B04F11E0359
:101500000B2220211846E662059303F0E2FB00203F
:10151000182384F829303146804602464FF0050EE4
:1015200016F9013B0D2B2FD01FDC8BB30A2B2BD0D0
:10153000D9B2202926D97E2900F2CE80964D05EB1E
:10154000030C1CF821CC1CF0210F00F09780B8F19F
:10155000000F17D01CF0200F14D0072A40F3A680EC
:10156000002800F0D1800A2A97E02F2B10D05C2BA6
:101570000ED02E2BDCD1002A00F09880082AECDC5B
:10158000012008223146CBE722B94FF0FF3305E0B6
:10159000002AF7D0B3FA83F35B090E46A361013347
:1015A00000F0DA81C4E90C6696F900305C2B01D0BA
:1015B0002F2B00D10136049A542353434FF00009D6
:1015C000099379680898FFF7EDFD8046002840F000
:1015D0002382099A6F4B13445B6902933B7A5B0148
:1015E0000393DDE902329D18B9F1000F40F05D81EF
:1015F000BBF1000F40F04A810C22394604F138005B
:1016000003F070FBDDE902329B5C069A002A40F091
:101610008C80E52B00F02781079B0193EB7A03F088
:101620003F020F2A00F09380DDE90210095C0029D7
:1016300040F08880082A0CBF6FF004096FF00109A0
:10164000082B09D0636C3BB9012363640B22294644
:1016500004F1480003F046FB636B2363019B002BFE
:1016600040F00681B9F1FF3F40F00281DDE902322E
:101670009B5C03F03F0B4FF00009D8E0B8F1000F7E
:101680007FF46BAF1CF0040F16D094F9291030B919
:1016900021F0080184F82910072A07DD34E021F041
:1016A0001001072A84F829103FF75DAF05994FF024
:1016B00000088B54013265E71CF0080F3FF44DAF72
:1016C000A1F120035BB294F9291010B941F008018F
:1016D000E0E741F01001E4E701F17F0C5FFA8CFCD8
:1016E000BCF11E0F04D92031C9B21C293FF64AAF04
:1016F000002A7FF432AF13F11B0FD7D1012284F8F7
:101700001EE090463EE71646324612F9013B0D2B8D
:1017100003D004DC0BB10A2BF5D104233EE72F2BB9
:1017200001D05C2BEFD1022338E743B12B7B33B9D7
:10173000AB7E23B9EB7E43B1CDF804906EE7CDF8D4
:1017400004B06BE76FF002097AE7079B0193DDE9CC
:101750000232985C10F0400C03D0636B23634FF0AF
:10176000010C0D2212F1FF3208D26B7BBCF1000F8D
:101770004ED194F85510994227D14BE0531E0B2BB4
:101780003CD8DFE803F039373533312F2D2B2927AB
:10179000250B00BF8005FF1F9B640000AB7F591E17
:1017A000C9B2FD29DED8216B01F1FF3EC4F830E05B
:1017B00011F8011C8B42D5D0A3F1410EBEF1190FD7
:1017C0001ED82033DBB28B42CCD04FF0FF3943E739
:1017D0002B7FE4E72B7EE2E7AB7DE0E72B7DDEE7C6
:1017E000AB7CDCE72B7CDAE7AB7BD8E76B7AD6E720
:1017F000EB79D4E76B79D2E7EB78D0E76B78CEE77B
:10180000A3F1610EBEF1190FDFD82031C9B2DAE7BA
:1018100084F8553000F03F000128D4E90B321DD187
:101820009A42D2D1636B2363019B83F001093B7A17
:101830007C4A09990133DBB20A443B72128DB3EB47
:10184000521FFFF4BEAE4FF000033B7239460898BA
:10185000FFF7E0FC00283FF4B4AE95E09A42B4D321
:101860004FF0000BE3E7069B01936FF00309F3E6EB
:1018700019F1030F76D019F1020F7FF4FCAE96F93F
:101880000030002B68D16FF0050867E0BBF1010B59
:10189000CDD1636C002BE3D1012363640B22294675
:1018A00004F1480003F01EFAE5E62A4605F10B01B3
:1018B00012F8013B03EB500303EBC0138A4203F021
:1018C000FF00F5D194F8553083424BD10123A36139
:1018D000A36923F00203012BA9D1DDE902329B5C4D
:1018E000002B42D0E52BA2D0EB7AB9F1000F08D142
:1018F0001B079CD40B220599284603F02EFB0028D9
:1019000095D12B7D6A7D1B0403EB0263EA7E03EB1A
:101910000223AA7E1344E360CAF80450EA7AD00690
:101920003FD4404A0498CAF82C30542101FB0021CE
:1019300091F82B20C868098B02FB03034904CAF8FD
:10194000303006D5012A04D9C2F101021A44CAF87E
:1019500030204FF0020801E06FF0020840460FB05F
:10196000BDE8F08F4FF00009B2E7626911070BD5AF
:10197000BAF83820AAF8363002F00102AAF8382066
:10198000DAF8002002B11370A369002BE4D0A38B16
:101990001A077FF578AF0C220BA9384603F0A2F99D
:1019A00071E7A26932B1A28BD20603D596F9002065
:1019B000002AD3D01B4904983B60542202FB00123A
:1019C00092F82B10D26803FB01237B6002233B7249
:1019D00096F900309BB96369022B20D01B07BDD557
:1019E0000AF1140421460C220AF1080003F07AF9E6
:1019F0000C2221460AF1200003F074F9AEE70C2214
:101A000039460BA803F06EF92660B9F1000F3FF4D8
:101A100075AD0423A36171E56FF003089EE74FF0F5
:101A200003089BE78005FF1F2DE9F04F4D4D06464B
:101A30002868ADF5057D002110F002008DF8071033
:101A400006D04948494B42691B689847441C6AD0F4
:101A50002B6813F0010740F01F83454C2368122BBD
:101A600030D8DFE813F013001300370041005700AF
:101A70009F00AD00BB00CE00D800F9003301430148
:101A800028015E018E019801C4018002394B3A4A57
:101A90001A60364B394A1A60394D01F0DDFE39487B
:101AA00039493A4A00236B7043704B705370AB70E6
:101AB00083708B7093700223012211464D202360A6
:101AC00003F0F6FB052202A9B07B02F0ABFF002871
:101AD000F8D128E02E4B1A6842F000621A601A68AA
:101AE0001101FCD40323E7E700220DF10701294887
:101AF00001F0EEFE20B1013015D000238DF8073043
:101B00009DF80730012B03D00020FFF7DDFBD9E75C
:101B10000423236004AA0DF107011F4801F0D8FE39
:101B200028B10130F0D10DF5057DBDE8F08F9DF8AD
:101B30000730012B13D19DF81330AA2BE4D19DF867
:101B40001230012B06D10523236004214D2003F020
:101B50007FFBB7E7114803F0DDF90120D5E7104816
:101B6000F9E700BF2405FF1F8005FF1F1405FF1FB5
:101B70002805FF1F1805FF1F19140000811300001E
:101B8000FF01FF1FF001FF1FF501FF1FFA01FF1FFB
:101B90002C100B40F9640000FF6400000964000091
:101BA0002164000000220DF10701BB4801F090FE06
:101BB0000028B6D19DF80730012BC6D80623236034
:101BC00004AA0DF10701B54801F082FE0028A8D152
:101BD0009DF91030002BB6DA07232360B04803F0DC
:101BE00099F99DF81030AF4A13F040031BBF402312
:101BF00013831383AC4808BFAC4803F08BF9082368
:101C0000236004AA0DF10701A94801F061FE002834
:101C100087D10923236004AA0DF10701A54801F02B
:101C200057FE00287FF47DAF9DF8123003F01F03AC
:101C3000052B0FD1A04D9848A049A14A9DF810301E
:101C40006B7043704B7053709DF81130AB708370A4
:101C50008B7093700A23236004AA0DF10701984842
:101C600001F036FE00287FF45CAF8E4D10220DEBA4
:101C7000020105F1380003F035F89DF810309DF8A9
:101C800017009DF818209DF8191013F0400F52D03E
:101C9000130203EB00430B4401339B022B61894881
:101CA00003F038F96B6923B94FF4007003F096F92B
:101CB00068610D23236004AA0DF107017F4801F03C
:101CC00007FE00287FF42DAF0B23236000220DF1C7
:101CD0000701714801F0FCFD00287FF422AF9DF858
:101CE0000730012B3FF631AF0C23236004AA0DF11E
:101CF0000701714801F0ECFD00287FF412AF0E23BC
:101D00002360684B704D93F83B30322B0CBF4FF47F
:101D100090704FF4807001F083FD2B6843F0020354
:101D20002B6004AA0DF10701684801F0D1FD0546BA
:101D3000E8B1451CF6E69DF816309B0203F44063BB
:101D400003EB800303EB921349009DF81A2001F086
:101D5000060101EBD2119DF815200133023102F08A
:101D60000F028B400A2A2B6199D15B0096E70F2363
:101D700004214D20236003F06BFA4A4B83F848504E
:101D8000A0E6484B00221A60FFF7DAFA421C3FF443
:101D9000CAAE10232360C31C02D1FFF7B7FA91E645
:101DA0001123236000287FF4AFAE3E494A6992F8C0
:101DB000C2010B46F0B192F9520046281AD092F9AE
:101DC0003600462816D092F8C83192F8C9011B0493
:101DD00003EB006392F8C70192F8C62103EB0023DE
:101DE00013440B60FFF7ACFA441C3FF49CAE033085
:101DF000D3D001E000221A602A4A5369D97D987D28
:101E000093F80C9010EB01204FEA09290ED193F8BA
:101E1000260093F82710000400EB016093F82510CA
:101E200000EB012093F8241001270844197DDC7C85
:101E300014EB01240DD193F8224093F823102404CD
:101E400004EB016493F8211004EB012493F82010B3
:101E50000C44D06193F810A082F82AA0597B82F834
:101E60002B1093F80FC093F80EE0D2F800800EEB21
:101E70000C2E1FFA8EFE08EB0E0CB9F5007FC2F88F
:101E800020C005D321B109FB01FBBBF5004F21DDCB
:101E90000F4803F03FF880E7F001FF1F0A650000DC
:101EA000466400008005FF1F546400006464000065
:101EB0000565000014650000FF01FF1FF501FF1F0D
:101EC000FA01FF1FE265000028100B400F650000BB
:101ED0006F64000000FB0AF0B2F818A0A2F8289086
:101EE0002AF0080A1FFA8AFA4AF0200BA2F818B062
:101EF0000EEB00094FF6F47BA4EB0909B9FBF1F9ED
:101F0000D94500F2AD80002F40F0AA80012757602C
:101F100003F1240793F93A30322B01D18B48B8E70B
:101F20004AF4804343F0200313835368A4EB0E0468
:101F3000241A6044906003FB1100138BB4FBF1F48E
:101F40005904D06044BF1F30D0605462F91D0B2289
:101F50007F4802F0C7FE7F4B12221A60FFF7F0F9AC
:101F6000431C3FF4E0AD7C4C00284CD1208B47044F
:101F700049D4636993F8FF21AA2A44D193F8FE213A
:101F8000552A40D1DA78412A3DD19A78612A3AD14E
:101F90005A78522A37D11A78522A34D193F8E72145
:101FA000612A30D193F8E621412A2CD193F8E5211A
:101FB000722A28D193F8E421722A24D193F8EA21D5
:101FC00093F8EB1193F8EF71120402EB016293F8AE
:101FD000E91102EB012293F8E8110A4493F8EE119B
:101FE0002263090401EB076193F8ED7193F8EC317A
:101FF00001EB07210B44023A934298BF40F00400E2
:10200000636398BF2083554802F084FF238B5448B4
:1020100043F080032383534C02F07CFF238FD907C6
:1020200016D594F83A80B8F1000F11D127683C22F8
:102030004146204602F04DFE0123238784F83A8072
:1020400037B127604849384602F095FF0323E386FD
:102050002B6843F001032B603E4B13221A6031E5DD
:1020600093F8317093F8309093F82FA009EB07297B
:1020700093F82E703F0407EB0A6793F82DA007EB47
:102080000A2793F82CA05744576018FA89F7D762AB
:10209000176003F1400748E7DA067FF513AD2E4AD3
:1020A000324FD2E9070439680444A14291463ED236
:1020B000641A0A2CDFF8C0A02D4D28BF0A2414F1A1
:1020C000FF34FFF442AD3968DAF8003022484A1C88
:1020D0000DF110083A60424698470028EFD1B9F850
:1020E00018302A6813F4804315D0034658F820109E
:1020F00041B90232012301308028F7D1002BDED014
:102100002A60DCE71FFA81FCBCF1000F01D0090C4A
:10211000F1D10132EEE7184658F8231009B901321F
:1021200001200133802BF7D10028C8D0E8E723F045
:1021300010032B600E4B0F4C1B681363BF2194F9E7
:10214000000002F0F7FE00232370BBE47C64000073
:10215000C905FF1F2805FF1F8005FF1F88640000B9
:10216000E26500004405FF1F976400003805FF1F6B
:102170003405FF1F1C05FF1F1405FF1F2DE9F04F3D
:1021800007469FB057F8043B93F83A608E4B5422B1
:102190000D4606FB0231044601914FF000084FF056
:1021A00064090391A1680198FEF7FCFF002840F044
:1021B0000881039B227B596952018B1811F802A0F8
:1021C000BAF1000F41D0BAF1E50F00F0EF80D97AF3
:1021D00001F03F0CBCF10F0F4A4640D1002A3ED01F
:1021E0001AF0400F38D0997F0139C9B2FD299FBF3D
:1021F0001EA909F1FF32891801F8640C93F80D80CB
:102200000D2A00F3A680002105A802F062FD00223D
:102210005FFA82F94FF0000A237B039A0133DBB2A5
:102220002373128DB3EB521FC0F0C58000232373BC
:1022300039460198FEF7EEFFC31D40F0BC80BAF1AD
:10224000010F08BF6FF00F0003E0DB7A1A07E3D439
:1022500001201FB0BDE8F08F587B4045D0D011F071
:10226000020A40F0A38011F00801D5D193F80CC008
:1022700005F10902029210460CF0080203F1FF3E3C
:1022800005F1110B16461EF8012F202A0ED0052A43
:1022900008BFE52236B1A2F1410ABAF1190F9CBF7D
:1022A0002032D2B200F8012B8345ECD11A7A202AD1
:1022B0001AD086462E220EF8042B03F1080A0130AC
:1022C0000CF0100C1AF8012B202A0DD0BCF1000FD5
:1022D00006D0A2F1410BBBF1190F9CBF2032D2B244
:1022E00000F8012B7045EDD100220270DA7A2A72D3
:1022F0009A7FD87F120402EB0062587F02EB002223
:10230000187F02442A60587E1A7E02EB0022AA80BF
:10231000D87D9A7DB9F1640F02EB0022EA8015D0D6
:1023200003F10B0013F8012B02EB510202EBC11178
:10233000834201F0FF01F5D1414537D105AB03EBF5
:102340000901029802F017FE4FF064094FF0010AEC
:1023500062E71EA91144987F01F8650C187F01F807
:10236000660C187E01F8670C987D01F8680C187DE2
:1023700001F8690C987C01F86A0C187C01F86B0C68
:10238000987B01F86C0C587A01F86D0CD87901F83B
:102390006E0C587901F86F0CD87801F8700C0D3A72
:1023A0001EA911445B7801F8643C31E74FF0000A44
:1023B0004FF0640930E7BAF1000F3FF4F3AE0020AC
:1023C00047E76FF0030044E78005FF1F2DE9F04F5A
:1023D00000220C46D1F800A04A81097DE28111F06B
:1023E000010FA7B00CBF2C232F2380460193202779
:1023F000E189A289914201D3002011E008F104058E
:102400000C22294602A802F06DFC0AA94046FFF7FB
:10241000B5FE814638B110F1100F04D06FF00E00F8
:1024200027B0BDE8F08F6689019B0DF131001E4495
:1024300002F0ADFD22893044904207D90C2202A956
:10244000284602F04FFC6FF00D00E9E7BDF82C5074
:10245000217DBDF82E309DF83020009305F01F0B34
:10246000C5F34316C8074FEA552505F2BC756275DA
:1024700040F19780D10643D412F0010F0CBF4FF406
:10248000D2724FF49272002164204FF02D0C93050C
:102490004CBF0AF801000AF801C0722833D077282F
:1024A0000CBF78207220013152000A2992B2EED17D
:1024B00074490AF10A0002F05EFD9DF8301011F037
:1024C0001001024621D0D8F800306F4993F83A3015
:1024D000542000FB0313002193F82B001B8D58435D
:1024E00002F03CFB0346023E01301F700A2E0ED85C
:1024F000DFE806F041434547494B4D4F51535500E6
:1025000040F2ED32BFE77720CDE70A98E8E75F4970
:1025100002F031FD60210246584602F01FFB2021E7
:102520000246284602F01AFB05466E1C30462F7004
:102530000DF1310102F01FFD227D861B120782463C
:10254000A67506D402460D2102F8021B0A2141702D
:1025500092462268AAEB02026281E2890132E2819C
:10256000227D130744BF00228AF8002019F1100FC2
:102570007FF43EAF52E74649CAE74649C8E74649B5
:10258000C6E74649C4E74649C2E74649C0E7464967
:10259000BEE74649BCE74649BAE74649B8E7464977
:1025A000B6E7D0074CBF52222D228AF800209DF8B2
:1025B000302091074CBF48222D228AF801209DF837
:1025C000302052074CBF53222D228AF802209DF85A
:1025D00030108B064CBF41212D210AF104028AF8EC
:1025E00003105846602102F0B9FA4FF02E0B421C3E
:1025F00080F800B04021304602F0B0FA0021421CC1
:1026000080F800B0284602F0A9FA009B0770421C2F
:102610006021D80A02F0A2FA3A230370009B421C00
:102620004021C3F3451002F099FA9DF83030DE06E0
:1026300005460AD5237DD90703D4204902F09BFC27
:102640000546238A013323826FE705AE32462021F7
:102650000A9802F083FA801BC0F1110028448542D9
:102660000CD12846314602F086FC638A0A9A01336F
:102670006382636813440546636056E705F8017B8F
:10268000EDE700BF196500008005FF1F256500000C
:10269000296500002D6500003165000035650000EA
:1026A000396500003D65000041650000456500009A
:1026B000496500004D65000051650000556500004A
:1026C00038B50A4C238F0D4673B90123238784F84C
:1026D0003A0039B1C81880B202F080FC206003488B
:1026E000A58638BD2160FAE70020FAE74405FF1F00
:1026F00030B597B005460C4658220021684602F0D6
:10270000E8FA22462946684600F00AF8049B23B1FD
:10271000002221466846FEF7CDFE17B030BD00000E
:102720002DE9F8430F461446944992F83A20542371
:1027300003FB02130546188B060640F11A8100239D
:102740006B61B7B1E68E97F900C0BCF12E0F0ED1C8
:1027500097F901C0BCF12E0F09D1D4F800C0BCF12B
:10276000000F63D1278F47F0400727876746002B6C
:1027700070D1238F2F6023F4FC76AB8326877FB143
:1027800097F900605FFA86FEBEF10D0F00F2B88087
:1027900042F2014C2CFA0EFC1CF0010F00F0B2804A
:1027A00001236B61AB8B13F0020F04F120062ED1D5
:1027B000542303FB02114B68EB60012B636191F81A
:1027C0002B70CA6800F2AF80410440F1AC80A2F1E6
:1027D0001F033B44A36104F11407002323770C2259
:1027E000394604F1080002F07DFA0C2239463046E1
:1027F00002F078FA072323876B69206843F0080307
:102800006B6120B15E4902F0B6FB0323E386AB8B1C
:1028100013F0E40F00F0A5805A0640F187800C22E7
:1028200004F10801304602F05DFA8FE0032E2ED944
:102830000BB1013EB6B21CF906E0BEF15C0F02D04E
:10284000BEF12F0FF5D197F902C00133BCF1000F93
:1028500020D10237238F032E43F0400CA4F838C058
:10286000A5F81CC03CD923684FF0000913F9068075
:1028700003F80690238F206823F010032387214656
:102880000330FFF735FF38B1236803F806806FF097
:1028900002001FE0033756E797F9003063B1AB8BB6
:1028A00023F0C00343F08003238721463846FFF717
:1028B0001FFF30B1A5F81C90AB8BDF050CD5E68669
:1028C00007E0AB8BDB0507D52068791E304402F0AA
:1028D00052FB0520BDE8F883236803F80680F9E77A
:1028E000DE057FF546AF23680022DA700323E38616
:1028F0000C2204F1080104F1200002F0F3F9E8E7EA
:102900005C2E02D02F2E7FF44DAF43F02003AB831B
:1029100097F901301BB15C2B01D02F2B01D104237F
:102920003FE702233DE707FB032353E71B060DD4D4
:102930006B6913F0060F4FF00C020FD004F1080181
:10294000304602F0CFF968690428C3D06E60686928
:1029500010F0050010D101232B61BBE704F1140135
:1029600060E704F1140169600C22304602F0BAF904
:10297000EDE76FF00100ADE70020ABE78005FF1F3A
:10298000976400002DE9F74300230386436890F81D
:102990003680DB0704460F4616464AD5D0E9023298
:1029A0009B1A03D1002003B0BDE8F0839E4200D9FA
:1029B0009EB2214B542208FB0239C8462AE0E36844
:1029C000E16AC3F30803C3F50075ADB2B54228BF91
:1029D000354613B9B5F5007F22D000953A464846F2
:1029E000FEF7F6FBC8B9E368228EB8F828102B442E
:1029F0002A44761BE3602286B3FBF1F201FB12331B
:102A0000B6B22F4433B904F128014846FEF702FC60
:102A10000028C8D1002ED2D1C4E76FF00300C2E76E
:102A200094F83620054B484653F822303A469847EA
:102A3000D8E76FF00800B6E78005FF1F1405FF1FF9
:102A400038B50C46096861B1FFF752FE051E06DB7A
:102A500020460C2250F8041B203102F043F928468E
:102A600038BD6FF01005FAE7024B542200FB02302C
:102A7000704700BF8005FF1F70B5064696B00C4634
:102A80001D460A60002A78D092F83A303E4A542116
:102A900001FB03231B8BD90602D515F0260F6FD13E
:102AA00058220021684602F014F923681A8F15F0A5
:102AB000200F14BF42F01C0242F00C021A8731466C
:102AC00022686846FFF72CFE049B0646002B3FD089
:102AD0002A4621686846FEF7EDFC022806463AD1F0
:102AE00020460C2250F8141B203102F0FBF820463F
:102AF000082250F8201B2C3102F0F4F8204608225E
:102B000050F8281B2C3102F0EDF821684B68DA7A76
:102B1000D20748BF25F0060565609A7FD87F12046A
:102B200002EB0062587F02EB0022187F0244A26091
:102B30000022E26091F83A2084F83620597C1A7C11
:102B400042EA01226286DA7B9B7B43EA0223A38668
:102B5000304616B070BD0028FAD120460C2250F83D
:102B6000141B203102F0BEF845F080052368656033
:102B700093F83A3084F83630EAE76FF00B06E7E76F
:102B80006FF01206E4E700BF8005FF1F2DE9F04F4C
:102B9000012A85B004460D46C36825D0022A30D0EC
:102BA000002A18BF00259D421CD094F836602FD211
:102BB000082204F1200104F1280002F093F8002318
:102BC000E3603E4B542206FB023AE368BAF828B0B1
:102BD000CBF1000909EA0308564605EA0909C1458F
:102BE0001BD8E560002066E0002904DA4A429A42D8
:102BF0000CD81D44D7E78268D21A914228BF1546E7
:102C0000F7E782688A4201D9551ACCE70025CAE75E
:102C1000A3689D4228BF1D46D3E7E36AB26896F8D1
:102C20002B100133E3629B1AB3FBF1F201FB123369
:102C300033BB328B376AA36A520423D507EB1327C1
:102C400039465046FEF7AEFA80BB94F8283002228F
:102C500000925B000DF10A0239465046FEF7B8FAC1
:102C600020BBBDF80A300393A26A736A9A4220D847
:102C7000039A96F82B30F168A26202FB0313E36219
:102C8000D844ACE707EBD31739465046FEF78AFA2B
:102C900060B9A36A042203F07F0300929B0003AA99
:102CA00039465046FEF794FA0028DDD06FF0030055
:102CB00001E06FF0060005B0BDE8F08F8005FF1F52
:102CC00070470000044B48F201021A80034B49F69A
:102CD00076021A80704700BF02200540FEFF0220E6
:102CE0000A4B0B491A680A6830B5002808BF012052
:102CF000783A0C68A24203D21D68ED03F9D51A6830
:102D00000138A4F17802F4D130BD00BF10E000E03A
:102D100018E000E072B6024A13680133136070478E
:102D2000EC05FF1F034A1368013B136003B962B649
:102D3000704700BFEC05FF1F08B5064B4FF000724F
:102D40001A60FFF7E7FF02F0E9FABDE80840FFF775
:102D5000E9BF00BF04ED00E0F8B51E4C236853B98D
:102D60001D4D1E4F37F8136025F8136001331E2BDD
:102D7000F8D11B4B23601B4B1D782D06FCD51D780D
:102D800015F0300F1CBF30251D70174B1870C31F76
:102D9000022B0FD8154B0D0C1D700D0A03F8015CAA
:102DA00003F8021C0728A3F1020301BF1168596050
:102DB00052689A600B4DFFF7ADFF2846236898478D
:102DC000FFF7B0FF2B7813F0310F14BF0120002064
:102DD000F8BD00BFE005FF1F0806FF1F0602FF1F2A
:102DE0000906FF1F000002400700024006000240E3
:102DF0002DE9F8439046384A384C1E46054613687C
:102E00000C276F433B44A3609B6813F0400F0BBF3C
:102E100006F1100306F11803636063600CBF06F14E
:102E2000140306F11C0308469146E360FFF772FFA6
:102E30002A4BD8F804102A4602F0FAFD032807D0DE
:102E400004281DD0012823D1FFF76CFFBDE8F883CB
:102E5000D4E901135A6842F080020A605A6882F08D
:102E600040025A609A6882F040029A60D8F80030B6
:102E700043F08003C8F80030FFF754FF0020E5E777
:102E8000D5B984233361B3610821284603F07EF865
:102E9000D9F80010CB199A68114B134022681343DC
:102EA0002360ADB9DA0013D583F0400242F080020E
:102EB000C8F80020CB51DFE7284603F075F8094B2E
:102EC0001B6803EB401384221A619A610821DDE735
:102ED00043F08002ECE700BF4406FF1F4806FF1FD7
:102EE0000800FF03F005FF1F2DE9F74FDFF804830B
:102EF000B34EC14698F8004033781C4000F05D8125
:102F000034F0080700F09180FFF704FFE2074CD58A
:102F100073233370AB4BDFF8E0A21A7842F0020261
:102F20001A7098F8002002F0CF0288F80020A64A14
:102F30001268916821F040019160802111601A7837
:102F4000A24902F0FD021A70A14A00231370012267
:102F50008AF800209F4A1370137113710B700B7164
:102F60000B720B730B740B750B760B77137182F866
:102F7000303082F8343082F8383053461D7815F0FE
:102F80000405FBD1944B954A1B68DFF85CB29A604C
:102F900040321A6029465B462A46042002F048FD6A
:102FA0000D238BF816508AF80030A30719D58C4BE7
:102FB0001A78D50641BF8B498A6801328A601A782F
:102FC000500741BF87494A6801324A601A78910721
:102FD00041BF84490A6801320A6016221A7002232E
:102FE0003370E2060DD53023337099F8003043F08A
:102FF000200389F8003000231A461946052002F004
:1030000017FDA3060DD53023337099F8003003F077
:10301000DF0389F8003000231A461946062002F023
:1030200007FDFFB2FFF77EFE377025077FF562AF21
:10303000DFF8C8E1684B9EF800009EF80020D3F846
:1030400000C0604F684D000901B212F0080F0CEB90
:10305000411326D03A7814071ED45B4A126801EB5C
:10306000410402EB8404AC60A268510614D403F15D
:1030700010026A601433EB60FFF74CFE5A4B0246B5
:103080000021032002F0D4FCFFF74CFE504BAA7D38
:103090001A70082333702DE703F118026A601C339D
:1030A000E9E72A6802F080542C609EF8002052075D
:1030B0001DD597F800E01EF0080F03F1080202D1B9
:1030C00044F040042C60141D2C611468C4F3094EB4
:1030D00004F03C04042CA5F814E00BD0342C30D0C0
:1030E00084221A619A61082102F050FFD1E71A4642
:1030F0003C78E8E7344C276801EB410507EB850C89
:10310000DCF808C01CF0080FDFF8ECC018BF57F857
:1031100025701CF8211014BF07F080078027C9060E
:103120004CBF01210221FFF763FE226852F82530CF
:1031300027B123F0800342F82530AAE743F080034B
:10314000F9E701EB4101DFF880A0019100241C6147
:103150009C61DAF80010019C01EB840E2349DEF833
:10316000084021402C6814F0400408BFCCF800103F
:1031700041F0C00B17BFCCF8081021461C49CCF811
:1031800000B029604FF0480108BFCCF808B0CEF875
:1031900004100021FFF72CFE012809D0DAF80020E6
:1031A000019B019952F8233043F0800342F821300B
:1031B0003B7803F0DF033B706BE703B0BDE8F08FB3
:1031C00080200740942007404406FF1FD02007407E
:1031D00098200740C4200740F005FF1F8800080022
:1031E00088200740D405FF1F4806FF1F0800FF0383
:1031F0004000001084200740C02007409020074076
:10320000104B1B684033090143F8202000F1604354
:1032100003F56443C9B2424219704FF0200390FB9A
:10322000F3F34FEA830302F01F0203F1604300F05F
:103230001F0003F5614358BF5042012202FA00F01B
:103240001860704708ED00E0084B094ADA63094A44
:10325000094B13605360D2F80C3D43F07043C2F841
:103260000C3D064B07221A60704700BF0000FF1F8D
:10327000392D000014E000E07F8D5B0010E000E0DD
:1032800008B5094B1B88DB070AD5FFF743FD074B41
:103290004AF202621A804BF280421A80FFF742FD26
:1032A000034B20221A6008BD002005400C20054079
:1032B0008CF00F40134B20F0800210B51C685101B8
:1032C000000604EB010313D50F49104C08680C21CC
:1032D00001FB0201486820F04000486000211961AC
:1032E000996114F8223023F0020304F8223010BD53
:1032F000625822F0040262509A6822F004029A6036
:10330000F5E700BFF005FF1F4406FF1FC020074080
:1033100038B5174B13F820305A0727D5154B1C68C2
:10332000154B1B680C2204EB401402FB00300B68A9
:103330009860FFF7EFFC83685B0657BF2069A069C0
:1033400004F1100504F1140244BF04F1180504F15E
:103350001C0210F0800003D0FFF7E4FC022038BD0F
:103360000B685D60DA60FFF7DDFCF8E70120F6E747
:10337000C0200740F005FF1F4406FF1F2DE9F04F56
:103380009C460F46464BDFF824B192461A681BF85C
:10339000273023F00C030BF82730424B07EB47088C
:1033A0001D6849014FEA8808561805EB080985B0E1
:1033B0000024FF28B4613461B460DDF838E0545073
:1033C000C9F80840994645F80840374B08D11A78A3
:1033D00002F0CF021A700BF8274005B0BDE8F08F5D
:1033E0001D7845F010051D7020F08003012B36D1AB
:1033F000D9F8005045446C604425000646D47068F6
:1034000090B9E24538BFE246BEF822C01CF0400F3A
:103410002DD0DEF808C0ACF81400DCF80000CCF8C1
:10342000080070605044F060DFF884C00CEA0A4A7B
:103430004AEA040444F0800C24F04004C6F808C0B2
:1034400044F080065650D9F80020904445F008001A
:10345000C8F80840FBB905460BF82750BDE7D9F876
:10346000004044440825656005254824C5E75046CA
:10347000CDE90221019301F0B1FD7060504601F0E9
:10348000ADFDDDE90221F060019BCDE7002BE3D02B
:1034900045F01005E0E705F0FB0545F01805DBE712
:1034A000F005FF1F4406FF1F84200740C02007408F
:1034B0000000FF031C4B2DE9F3411D681B4F04B2B4
:1034C00005EB441504EB4404A4003A681259530672
:1034D00054BF08354FF000082A6858BF4FF0400825
:1034E00012F080061BD100960123C2F309426968DD
:1034F00002F004FA012814D039680B1930469A6892
:103500000B4B134043EA080343F080022A600A5938
:1035100002F0800213430B5102B0BDE8F08101209C
:10352000FAE70220F8E700BFF005FF1F4406FF1F7F
:103530000800FF032DE9F74F644A4C7C136843F4FD
:103540008073136002F52032043213680D4643F095
:1035500080735F4913600B6843F000430B60106891
:1035600023F0804340F0007010600B602B7C01342E
:10357000012BE4B2574B40F096801A6842F4E022E7
:103580001A6000225A64544B544E0022102C1A60C8
:1035900028BF1024524B012204EB44001A60800023
:1035A00001F01CFD4F4A1060337843F08003337004
:1035B000914633781806FCD46B89590705D44A4BD9
:1035C00002221A70802203F8042C484F02233B7019
:1035D0004FF40071600101F025FD454B454A18602C
:1035E000000A107059881175D97811764249002265
:1035F0000A703A7028310A7098468A469AF8003064
:103600005A07FBD46B8913F0040F14BF402408241D
:103610001FFA84FBD8F800300193584601F0DEFC15
:10362000019B5860D8F800300193584601F0D6FC51
:10363000019BD8F80020D860230443F088019160F2
:1036400043F0C8011160D9F8002043F008039360EB
:10365000802313600D238AF80030284BED221A7066
:10366000FF2283F87020BF2283F878200421244AA7
:103670003520FFF7C5FD6B8913F0040310D1214AF3
:103680001370214B8B221A7006221A7201233B7091
:103690006B89DB0704D5402333701C4B10221A7052
:1036A00003B0BDE8F08F1A4901220A6019494FF4AE
:1036B0000070086018490A60184A4FF4E061116010
:1036C0001A6822F480221A605DE700BF00F0014012
:1036D000007004400480044000D000400C210740EA
:1036E000C80690424406FF1F44210740942007402B
:1036F000F005FF1F9C20074098200740102007403E
:10370000E92E0000002107408420074008210740DF
:1037100024079042149004403407904268D004403B
:10372000002211464420FFF717BB000070B5C0F31C
:103730000B0520F47F64144E0D4424F00F04C4F3F1
:10374000120282B9B5420ED921460820FFF704FBC8
:10375000B8B9B5F5002F01D1002070BD04F50024E3
:10376000A5F50025EBE7002221460920FFF7F4FA32
:1037700038B9B5F5805FEFD904F58054A5F58055CB
:10378000DDE74FF0FF30E8E7FFFF07002DE9F84FD6
:1037900090468946204D89BB2B685A072BD023F0D1
:1037A00007032B600824DFF874A00AF1080BC4F1AA
:1037B0000806464528BF46460AEB040749463846F0
:1037C0003246374401F08EFA5F45B144A8EB060853
:1037D0001AD3524629680720FFF7BEFA0446B8B943
:1037E0002B6808220833FF2150462B6001F071FA44
:1037F000B8F1000FDBD10020BDE8F88F20F00703FF
:103800002B6000F00704CEE72B681E442E60EFE724
:103810004FF0FF30F0E700BFF405FF1FF805FF1F72
:1038200038B50B4C226822F00802226040F4602276
:103830002260084A054613681B07FCD545F460253D
:10384000322045F00805FFF74BFA256038BD00BF70
:103850002C100B4024100B40194A1A4808B540F2AE
:10386000434101231360C2F8F0300160C2F8F03028
:1038700040F8081CC2F8F03040F80C1CC2F8F030D8
:103880008160C2F8F0304160C2F8F0300E4B4FF466
:1038900088621A6003F5C823B83300221A604FF01B
:1038A000801243F87C2C202243F8982C4FF40150CE
:1038B000FFF7B6FF054B4FF0FF321A6008BD00BF9F
:1038C000440690420CD0044008D0044030100B4015
:1038D000F8B5704D704E2C6842F210739C420FDDAB
:1038E0006E4801F017FB6FF001042B682BB100212B
:1038F0004D2001F0ADFC00232B600023336099E0E4
:103900003368B3B9664F3B6813F0010CFBD1D0F8B4
:103910000130644F1BBA3B600378092B07F10407A1
:103920002BD00AD8D3B1022B27D01B0643F4D013D7
:1039300016E0062B15D00024D7E7112B21D0182B29
:10394000F3D1594BC3F800C04FF4813CC3F804C015
:1039500090F800C0554B43EA0C6301E04FF400338C
:103960003B60DFF868C1DCF8003013F0010FE64679
:1039700077D0037873B901230FE01B0643F4C81313
:10398000EEE7494BC3F800C04FF4813CC3F804C0D4
:10399000474BE5E7182B3BD100230B70454BCEF886
:1039A0000030002A74D00178434B092901D0022944
:1039B00062D142490868000C10700868000A507013
:1039C000096891703E490868000ED0700868000CC4
:1039D00010710868000A50710968917139490868C6
:1039E000000ED0710868000C10720868000A50724E
:1039F000096891721968090ED1721968090C11735E
:103A00001968090A51731B6893730024D4736CE717
:103A1000DCF8007017F480370ED02B4BCCF8003058
:103A20000134002301214D202C60336001F010FC93
:103A30004FF0FF342046F8BDDCF80040A40305D564
:103A4000292B01D10F70A9E70823A6E7DCF8004075
:103A500014F44024A2D1082B8DD0372B8BD00C70BE
:103A60009CE7062333601CB901214D2001F0F0FBD7
:103A70002B6801332B60DBE71968090E1170196898
:103A8000090C51701968090A91701B68D37052E7CC
:103A900014462AE7E805FF1FE405FF1FD86500006C
:103AA00024100B4008100B4000100B4026003A0079
:103AB00014003A1101000F0010100B401C100B40B5
:103AC00018100B4014100B4001000D0030100B407B
:103AD00010B519490A460B6803F08403042BFAD089
:103AE00016490B6801330B6015494FF47A7314685B
:103AF000240510D5134900F50073984217D1104BD7
:103B000019461868800702D410688407F9D50E4B4F
:103B10000B60002010BD0C6814F4E00F04D00B4BB8
:103B20000B606FF00300F5E7013BE0D1F9E70C68AB
:103B300040F8044BE1E700BF24100B400406FF1FD0
:103B400030100B4020100B402200000120007000BC
:103B5000F0B50D460B490B68ADF5017D0133064606
:103B6000684617460B60FFF7B3FF044628B97A1B77
:103B70000DEB0501304601F0B5F820460DF5017D4D
:103B8000F0BD00BF0006FF1F00F580204930002A6D
:103B900030B54FEA003018DA22F07F4222F470028A
:103BA00022F4FF420A4D22F07C020124ED4309E099
:103BB000214205D003682B401343036021EA04012E
:103BC000043064000029F3D130BD024DEDE700BFA1
:103BD00003000F0077070F00014B024A1A60FEE74F
:103BE0000CED00E00400FA0510B5114A1149124825
:103BF000891A002399420BD11049114A91420BD1E5
:103C0000104A11490023891A18468B420DD110BD64
:103C10001C5CD4540133EDE70C480023801A984211
:103C2000EED0CC5CD4540133F9E7D0540133ECE747
:103C3000F001FF1F9902FF1F28660000100400001A
:103C4000100400009C02FF1F9808FF1F5460000032
:103C50005149524C524808B501230B602268514B20
:103C600022F006022260504A106002F5342210321F
:103C7000084612684CF2205112F0040F4DF628123B
:103C800019801A8000F083804FF4C87223F8082C42
:103C9000002223F80A2C40F2D11223F80E2C012323
:103CA00003604FF4A27220210220FFF76DFF3F4A0C
:103CB000136843F020031360236843F0200323605C
:103CC0003B4B1B78802B02BF3A4B00221A703A4BB9
:103CD000A4221A70A02203F8012C05331A46197881
:103CE0008C07FCD51378D806FCD4137803F00C03AA
:103CF000082BFAD1314B21221A704E225A7002330E
:103D00001A4619788906FCD513785B06FCD52C4B2E
:103D10004FF08A721A602B4B28221A702A4A1378A5
:103D200003F00C030C2BFAD1284B294A9A61C3E902
:103D30000222C3E904221A639A63DA62254A1360F5
:103D4000FFF752FF244A136843F470031360002105
:103D50001620224AFFF754FA214B4FF480621A6072
:103D6000204A6FF07F43136053601F4B1A6805228F
:103D70001A60FCF7E7FE1D491D4801F011F9062203
:103D80001C491D4801F074F901F02EFAFCE71B4BA9
:103D90004FF4E9721A8082E72C07904294F00F40AA
:103DA000030106000E20054080B0044080F00F4063
:103DB00003E0074001E007400140064004400640A0
:103DC0004480044000400640064006400000FF1FBB
:103DD000C12C000008ED00E088ED00E0C52C0000DB
:103DE0000080004014E000E010E000E09808FF1FB1
:103DF00070650000676500007865000000200540E0
:103E0000D0F800D0D0F804F07047000070B5054637
:103E1000EBB2012B0846114653DC15F4406F0ED06F
:103E2000820751D1C0291FD0B1F5807F22D08029CF
:103E30004DD14FF48272274C5A430A26A65015F4EE
:103E400080641DD04FF482745C43224D04F114024F
:103E50002A4400F0DDF9201D10220021284400F042
:103E600038FF0024204670BD4FF482725A43194C2B
:103E70000C26E3E74FF482725A43164C0E26DDE718
:103E800015F400660FD04FF482755D43114E05F1B5
:103E90001402324400F0BCF9281D1022214630449F
:103EA00000F017FFDEE715F40054DBD0094A4FF4A9
:103EB000827101FB032301461022181D00F012FF3E
:103EC000CFE74FF0FF34CDE76FF00304CAE76FF0A0
:103ED0000404C7E76406FF1F2DE9F04F9B4687B037
:103EE000C3B2012B82460C461546019300F3808134
:103EF00010F4407F00F07F81019ADFF808834FF4CF
:103F00008273534358F80320002A00F07781294335
:103F100003F1040910F4807F01F0030108EB0906A6
:103F200000F0818049B15A460021284600F0D1FEB8
:103F30006FF0030007B0BDE8F08FBBF10F0F01D8A1
:103F40000020F7E710F4805F21685CD02960626888
:103F50006A60A268AA60E268EA6003F11407019B44
:103F6000A84A4FF4827A0AFB03FA17442B4652F808
:103F70000A202846394600F00BFC2B6848F8093027
:103F80006B687360AB68B360EB68F360ABF1100310
:103F900023F00F039B4A04F110081C441035203411
:103FA000924408F1100844452B4605F11005C7D08E
:103FB000316858F8102C4A4045F8102C716858F8B0
:103FC0000C2C4A4045F80C2CB16858F8082C4A4093
:103FD00045F8082CF16858F8042C4A4045F8042CA0
:103FE0001846DAF80020394600F0D2FB55F8103CAC
:103FF000336055F80C3C736055F8083CB36055F8D5
:10400000043CF360CDE758F809204A402A60716803
:1040100062684A406A60B168A2684A40AA60E26881
:10402000F1684A4098E700297FF47DAFAC4273D134
:10403000BBF10F0F84D9D4E90071143303914344C9
:10404000A16802930491E1680591234602992046F4
:1040500000F036FC1AF4805F10D158F8092023686C
:10406000534023607268636853406360B268A3681A
:104070005340A360F268E3685340E360039B48F851
:1040800009707360049BB360059BF360ABF1100390
:1040900023F00F0305F110071D44019BDFF8649125
:1040A0004FF4827A103405F120080AFB03FA3B46EC
:1040B0001037B845204604F110043FF441AF54E9ED
:1040C00004B2019254F8082C0392029959F80A207C
:1040D00054F8045C00F0F4FB326857F8103C53408D
:1040E00047F8103C726857F80C3C534047F80C3CBA
:1040F000B26857F8083C534047F8083CF26857F854
:10410000043C534047F8043C019B7360039BC6F892
:1041100000B0C6E90235CAE7BBF10F0F7FF610AF5A
:1041200003F1140747442B463946204600F0C8FBEC
:104130001AF4805F10D158F809202B6853402B6087
:1041400072686B6853406B60B268AB685340AB6099
:10415000F268EB685340EB60236848F80930636805
:104160007360A368B360E368F360ABF1100323F0FE
:104170000F0305F1100820351D44019B1A46214B01
:104180004FF4827A10340AFB023A434608F11008D1
:10419000A845204604F110043FF4D2AEDAF800201E
:1041A000394600F08DFB326858F8103C534048F80F
:1041B000103C726858F80C3C534048F80C3CB2680C
:1041C00058F8083C534048F8083CF26858F8043C5A
:1041D000534048F8043C54F8103C336054F80C3C0D
:1041E000736054F8083CB36054F8043CF360CCE7C7
:1041F0004FF0FF309EE66FF005009BE66FF0010088
:1042000098E600BF6406FF1F0000000000000000E9
:104210002DE9F05F40F22028C1F6FF78F0C824BAFB
:104220002DBA36BA3FBAF0C298E8001C802900F0D7
:10423000D781C02900F0FF8090E80A0309BA1BBAB1
:1042400098FA88F899FA89F9A2E80A035AF8040B4F
:104250004FEA396ECCF844E8CCF800B0DCF884E8DA
:104260008EEA000E84EA0E0485EA040586EA050655
:1042700087EA0607F0C2CCF84478CCF800B0DCF846
:1042800084E881EA0E0183EA010388EA030889EAE7
:104290000809A2E80A035AF8040B4FEA396ECCF871
:1042A00044E8CCF800B0DCF884E88EEA000E84EA3A
:1042B0000E0485EA040586EA050687EA0607F0C2C9
:1042C000CCF84478CCF800B0DCF884E881EA0E0140
:1042D00083EA010388EA030889EA0809A2E80A03D5
:1042E0005AF8040B4FEA396ECCF844E8CCF800B029
:1042F000DCF884E88EEA000E84EA0E0485EA040500
:1043000086EA050687EA0607F0C2CCF84478CCF8BE
:1043100000B0DCF884E881EA0E0183EA010388EA50
:10432000030889EA0809A2E80A035AF8040B4FEACD
:10433000396ECCF844E8CCF800B0DCF884E88EEABA
:10434000000E84EA0E0485EA040586EA050687EA7B
:104350000607F0C2CCF84478CCF800B0DCF884E86A
:1043600081EA0E0183EA010388EA030889EA080961
:10437000A2E80A035AF8040B4FEA396ECCF844E875
:10438000CCF800B0DCF884E88EEA000E84EA0E0473
:1043900085EA040586EA050687EA0607F0C2CCF836
:1043A0004478CCF800B0DCF884E881EA0E0183EAB6
:1043B000010388EA030889EA0809A2E80A035AF80F
:1043C000040B4FEA396ECCF844E8CCF800B0DCF8C6
:1043D00084E88EEA000E84EA0E0485EA040586EA83
:1043E000050687EA0607F0C2CCF84478CCF800B09E
:1043F000DCF884E881EA0E0183EA010388EA030815
:1044000089EA0809A2E80A035AF8040B4FEA396E50
:10441000CCF844E8CCF800B0DCF884E88EEA000E72
:1044200084EA0E0485EA040586EA050687EA06079B
:10443000F0C2BDE8F09F90E8000398FA88F899FA76
:1044400089F9A2E800035AF8040B4FEA3963CCF863
:104450004438CCF800B0DCF8843883EA000384EAFE
:10446000030485EA040586EA050687EA060788EA62
:10447000070889EA0809A2E8F0035AF8040B4FEA92
:104480003963CCF84438CCF800B0DCF8843883EADF
:10449000000384EA030485EA040586EA050687EA40
:1044A000060788EA070889EA0809A2E8F0035AF82B
:1044B000040B4FEA3963CCF84438CCF800B0DCF890
:1044C000843883EA000384EA030485EA040586EA63
:1044D000050687EA060788EA070889EA0809A2E8C4
:1044E000F0035AF8040B4FEA3963CCF84438CCF89F
:1044F00000B0DCF8843883EA000384EA030485EA28
:10450000040586EA050687EA060788EA070889EAB5
:104510000809A2E8F0035AF8040B4FEA3963CCF813
:104520004438CCF800B0DCF8843883EA000384EA2D
:10453000030485EA040586EA050687EA060788EA91
:10454000070889EA0809A2E8F0035AF8040B4FEAC1
:104550003963CCF84438CCF800B0DCF8843883EA0E
:10456000000384EA030485EA040586EA050687EA6F
:10457000060788EA070889EA0809A2E8F0035AF85A
:10458000040B4FEA3963CCF84438CCF800B0DCF8BF
:10459000843883EA000384EA030485EA040586EA92
:1045A000050687EA060788EA070889EA0809A2E8F3
:1045B000F0035AF8040B4FEA3963CCF84438CCF8CE
:1045C00000B0DCF8843883EA000384EA030485EA57
:1045D000040586EA050687EA0607F0C2BDE8F09FF3
:1045E000DAF800004FEA3763CCF84438CCF800B072
:1045F000DCF8843883EA000384EA030485EA0405CE
:1046000086EA050687EA0607F0C2DAF804004FEAF0
:104610003763CCF84438CCF800B0DCF8843883EA4F
:10462000000384EA030485EA040586EA050687EAAE
:104630000607F0C2DAF808004FEA3763CCF84438CE
:10464000CCF800B0DCF8843883EA000384EA030481
:1046500085EA040586EA050687EA0607F0C2DAF865
:104660000C004FEA3763CCF84438CCF800B0DCF8E3
:10467000843883EA000384EA030485EA040586EAB1
:10468000050687EA0607F0C2DAF810004FEA37633A
:10469000CCF84438CCF800B0DCF8843883EA000366
:1046A00084EA030485EA040586EA050687EA060724
:1046B000F0C2DAF814004FEA3763CCF84438CCF88B
:1046C00000B0DCF8843883EA000384EA030485EA56
:1046D000040586EA050687EA0607F0C2DAF818003C
:1046E0004FEA3763CCF84438CCF800B0DCF88438B3
:1046F00083EA000384EA030485EA040586EA0506E2
:1047000087EA0607F0C2DAF81C004FEA3763CCF8F4
:104710004438CCF800B0DCF8843883EA000384EA3B
:10472000030485EA040586EA050687EA0607F0C25F
:10473000DAF820004FEA3763CCF84438CCF800B000
:10474000DCF8843883EA000384EA030485EA04057C
:1047500086EA050687EA0607F0C2DAF824004FEA7F
:104760003763CCF84438CCF800B0DCF8843883EAFE
:10477000000384EA030485EA040586EA050687EA5D
:104780000607F0C2BDE8F09FAFF30080AFF30080F2
:104790002DE9F01F90E8F00024BA2DBA36BA3FBADE
:1047A00040F23020C1F6FF70B1E8000F84EA08043F
:1047B00085EA090586EA0A0687EA0B0790E8011FE1
:1047C0008BE8F000CCF80000CCF80080F0C989E854
:1047D000F000CCF80000CCF80080F0C989E8F000C7
:1047E000CCF80000CCF80080F0C989E8F000CCF8E3
:1047F0000000CCF80080F0C989E8F000CCF8000097
:10480000CCF80080F0C989E8F000CCF80000CCF8C2
:104810000080F0C989E8F000CCF80000CCF80080F6
:10482000F0C989E8F000CCF80000CCF80080F0C9AD
:1048300089E8F000CCF80000CCF80080F0C989E8E5
:10484000F0000A2A1DD0CCF80000CCF80080F0C996
:1048500089E8F000CCF80000CCF80080F0C989E8C5
:10486000F0000C2A0DD0CCF80000CCF80080F0C984
:1048700089E8F000CCF80000CCF80080F0C989E8A5
:10488000F000CCF80000CCF800809AE8F00091E845
:10489000000F84EA080485EA090586EA0A0687EA21
:1048A0000B0724BA2DBA36BA3FBA83E8F000BDE848
:1048B000F01F7047AFF30080AFF30080AFF30080CC
:1048C0002DE9F01F90E8F00024BA2DBA36BA3FBAAD
:1048D00040F25020C1F6FF7001EB021191E8000F89
:1048E00084EA080485EA090586EA0A0687EA0B07CE
:1048F00090E8011F8BE8F00031E9F000CCF80000EF
:10490000CCF8008089E8F00031E9F000CCF8000034
:10491000CCF8008089E8F00031E9F000CCF8000024
:10492000CCF8008089E8F00031E9F000CCF8000014
:10493000CCF8008089E8F00031E9F000CCF8000004
:10494000CCF8008089E8F00031E9F000CCF80000F4
:10495000CCF8008089E8F00031E9F000CCF80000E4
:10496000CCF8008089E8F00031E9F000CCF80000D4
:10497000CCF8008089E8F00031E9F000CCF80000C4
:10498000CCF8008089E8F0000A2A21D031E9F00053
:10499000CCF80000CCF8008089E8F00031E9F000A4
:1049A000CCF80000CCF8008089E8F0000C2A0FD089
:1049B00031E9F000CCF80000CCF8008089E8F00084
:1049C00031E9F000CCF80000CCF8008089E8F00074
:1049D000CCF80000CCF800809AE8F00031E9000F34
:1049E00084EA080485EA090586EA0A0687EA0B07CD
:1049F00024BA2DBA36BA3FBA83E8F000BDE8F01FFA
:104A0000704700BF08B5054B187000EB80008000B0
:104A100000F0E4FA024B186008BD00BF6C08FF1FED
:104A20007008FF1F13B5074C0138C3B2246803EBAD
:104A3000830004EB8004207C009364680423A04777
:104A400002B010BD7008FF1F70B50B4B1A680B4BFE
:104A50001D780024E3B29D4201D8002007E056688B
:104A6000864205D1167C8E4202D1581CC0B270BD60
:104A700014320134EEE700BF7008FF1F6C08FF1FFF
:104A80002DE9F84F81461046884617469A46FFF7AB
:104A9000DBFF014618B100263046BDE8F88FFFF76E
:104AA000D3FF06460028F6D01C4A14256FF01303E6
:104AB00015FB003315681D44B9F800309BB1504612
:104AC00000F08CFA0446A86068B1B9F800B0584606
:104AD00000F084FA0028DED0C4E90000A060584449
:104AE000E060A4F816B0B9F802309BB1504600F06F
:104AF00075FA0446E86068B1B9F80290484600F0DB
:104B00006DFA0028C7D0C4E90000A0604844E06006
:104B1000A4F816906F6085F81080BDE77008FF1F3D
:104B2000032807B503D0052811D000200CE0138915
:104B3000ADF804301168084A0023ADF80630097852
:104B4000182301A8FFF79CFF03B05DF804FB104693
:104B500000F066FEF8E700BF6D4D00002DE9F04F54
:104B60008F0641BF202301F0F701137001324E0779
:104B700005D50028BFBF2D23137040420132002508
:104B8000324B334C2E4601F0400801F008094FF03B
:104B9000200A68B337464FF0300C05E0E5B182F8E3
:104BA00000C03A4637467346834254F827E006F180
:104BB000010602F10107F1D8B0FBF3FC002B0CF168
:104BC000300B5FFA8CFC82F800B003FB1C0018BFAE
:104BD00001253A467346DCE7BEF1010FE2D1B8F198
:104BE000000FDCD1B9F1000FDCD082F800A0D8E7CB
:104BF00004EB8604043C302610466BB13DB90D072A
:104C000002F1010319D520201070184606E054F86F
:104C1000043F02F8016BEFE7002DF0D00B0606D53C
:104C200003460D2203F8022B0A224270184611F0A7
:104C3000100108BF0170BDE8F08F4C0642BF302064
:104C400010701846302303700130E7E700CA9A3B22
:104C5000FC650000F0B58C0642BF202313700132C2
:104C60000B0706D51346302403F8024B7824547002
:104C70001A4601F0100501F040074EB201F007019D
:104C8000042928BF0421490096460C46013CE4B2A1
:104C9000FF2C0BD1002E02EB010004DA0D2353543C
:104CA0000A234370023005B90570F0BDA30020FA55
:104CB00003F303F00F0303F1300CBCF1390F02D9F9
:104CC00027B103F1370C0EF801CBDFE703F1570CE6
:104CD000F9E7C9B202440346934200D1704703F892
:104CE000011BF9E710B5431E0A44914200D110BDE3
:104CF00011F8014B03F8014FF7E72DE9F843058A56
:104D0000954228BF154604460F460DB3D0F80480DF
:104D1000C66808EB0503B34243601ED3A6EB080642
:104D2000B6B20368A5EB06094B444360FDF7FAFFF2
:104D30004FB1324641463846FFF7D4FF21684A4614
:104D4000B819FFF7CFFFFDF7E5FF238A5B1B23822E
:104D5000FDF7E8FF2846BDE8F883FDF7E3FF002FE5
:104D6000F1D02A4641463846EBE70000F8B51D462B
:104D70000F4B9DF818001C6800EB800004EB8000CE
:104D80000E4617468468FDF7C5FF042D06D0052D95
:104D90000BD1248AFDF7C6FF2046F8BD3A463146BE
:104DA0002046BDE8F840FFF7A8BF0024F2E700BFA7
:104DB0007008FF1F2DE9F041044616460F46FDF727
:104DC000A9FF628A238AE18AD4F8088098183044BF
:104DD0008842C2BFCE1AB61AB6B2E36808EB06051F
:104DE0009D4228BF2368A56021BF6D1AA560ED1AFA
:104DF000751B32442CBFADB235466282FDF792FF7F
:104E00002A4639464046FFF76DFFAE4204D0721B7A
:104E100079192068FFF766FFFDF77CFF628AA18A97
:104E2000B2420BD1238A33440B4423820023A38252
:104E30006382FDF777FF3046BDE8F0817318921B5F
:104E4000A3826282F5E70000F8B5027843789A42BF
:104E500005460F4621D1867812483146FFF7F4FD0A
:104E6000E8B16FF01303142414FB00340E4B1868E0
:104E7000EB782044032B806805D1C48A008A241A69
:104E8000A4B22046F8BD29463A46FFF793FF042115
:104E9000044670B200F0DCF9F3E70024F1E70446C1
:104EA000EFE700BF6D4D00007008FF1F13B50B4604
:104EB00030B91146184602B0BDE81040FFF7C4BF34
:104EC000FF280ED0084C0138C3B2246803EB8300DE
:104ED00004EB8004207C009364680323A04702B0A5
:104EE00010BD0020FBE700BF7008FF1F10B4034691
:104EF00008461946CA1A11F8014B92B2002CF9D192
:104F000022B119465DF8044BFFF7D0BF10465DF89B
:104F1000044B7047014B1978FFF7E8BF9802FF1F59
:104F20001FB56A46FFF796FE6846FFF7F3FF05B028
:104F30005DF804FB07B568B10023ADF800308DF8CB
:104F4000020001238DF80410684605218DF8033016
:104F5000FFF77AFF03B05DF804FB10B50A449142F5
:104F600001D1002010BD10F8014B11F8013B9C420B
:104F7000F5D00120F6E70139034611F9012F184653
:104F800003F8012B91F90020002AF6D17047024660
:104F90000346981A13F9011B0029FAD17047000043
:104FA00010B50A4B00221A80094B0A4A19600A4BB5
:104FB000147819600278A24203D142881144196022
:104FC00010BD002AFCD00430F4E700BF7408FF1FB6
:104FD0007808FF1F0402FF1F7C08FF1FF8B50E4F63
:104FE0000E4E3C6831880E4A0C44A3071CBF24F0C7
:104FF00003040434126823189A4205460AD902466B
:1050000000212046FFF765FE3B68E31A1D4435800A
:105010002046F8BD0024FBE77808FF1F7408FF1F37
:105020007C08FF1FF8B50F4F0F4E3C6833880F4ABE
:105030001C444B1E1C421EBF4B421C40641812688D
:1050400023189A4205460AD9024600212046FFF756
:1050500040FE3B68E31A1D4435802046F8BD00241D
:10506000FBE700BF7808FF1F7408FF1F7C08FF1FC5
:105070002DE9F84F584B594F904600221A603A607C
:10508000574A12788246994691F9004014B925464C
:10509000264618E0E4B294426ED10D466E1A15F918
:1050A000014FF6B2002CF9D106EB860080000430E7
:1050B000FFF794FFF14329443860254611F9013F79
:1050C000002B56D103603B684BB3EDB105EB4500B7
:1050D0008000043080B2FFF781FF00213A68C9F8F0
:1050E00000008C464FF0010E4FF6FF7A1368002B3C
:1050F00049D109B1C9F80000D9F8003005EB4505E0
:10510000A3EB8505C9F8005004EB0800C0B2FFF717
:1051100079FC24B13C68FF252368002B4ED1314B2C
:1051200000221A60FEF790F83046BDE8F88F103282
:10513000D2F800C0BCF1000FC0D09CF900E09E4541
:10514000F5D15368C0E900C3138903810BB1013461
:10515000E4B2B2F80AC09389A0F80AC08381927BB6
:10516000C273BCF1000F00D10BB10135EDB21430A8
:10517000A4E75246DCE7014691F90130481C002BB8
:10518000F9D1023180E753899BB1534508BFA2F89A
:105190000AC0538943604FF0010B43680BB180F89C
:1051A00009E0BBF1000F02D040F80C2B01211432B2
:1051B0009CE79389002BEDD19B46EEE7238933B121
:1051C000224601210320FFF7ABFC10B1A073143479
:1051D000A2E7A573FBE700BF8408FF1F8008FF1F3D
:1051E0000402FF1F8808FF1F184B37B51C680025F5
:1051F00023680BB903B030BDE37B13F00D0F22D051
:10520000FDF788FDA38913B9E37BDB0716D4237C64
:105210007BB1ADF80050226812788DF80220694603
:10522000052200208DF803508DF80430FFF73EFE74
:105230002574E37B13F00A0308BFE373FDF772FDE7
:105240006368204698471434D2E700BF8008FF1FE8
:1052500038B5144B1C6823686BB193F90030834256
:105260001ED111B9104B1D683DB94A0702D5E37B29
:105270001B0700D4E17338BD0C352B68002BF4D02C
:10528000A342F9D1FDF746FDA3891BB1074A126875
:1052900013446B600023E373BDE83840FDF742BD63
:1052A0001434D8E78008FF1F8408FF1F8808FF1FF9
:1052B000F8B5174B1C680E4617464CB1154B1D68C8
:1052C0002B682BB193F9003083421FD1236803B9B7
:1052D000F8BDAB4218D1FDF71DFDEB7B23F00203B7
:1052E000EB73277237B9AE813EB96672BDE8F840FC
:1052F000FDF718BD002E08BF0126074B19680123D2
:105300000E4466606372F1E70C34DFE71435D7E7CB
:105310008408FF1F8008FF1F8808FF1F154A164BCF
:1053200011681B68013130B51160114623B10C338F
:10533000042553F80C2C02B930BD13F8030C98B1B6
:1053400053F8080C0C68A0420ED1D47B14F0020F65
:1053500005D1240758BFD57313F8044C14749289EF
:1053600022B1024443F8082C0C33E2E703F8032C83
:10537000FAE700BF8808FF1F8408FF1F40B1836958
:1053800093F82820501C83F8280003EB4203D983AC
:105390007047022910B500F1020408D011460378C5
:1053A00021F8023B407843EA002313800A46237821
:1053B0001380617843EA0123138010BD2DE9F8437F
:1053C0001F46354B1B682C2404FB07340646638BB1
:1053D000002B5ED1258BA2838A4228BF0A469542C4
:1053E000628328BF15469046089AE582D368DFF8A5
:1053F000AC901860D2E90103596809EA054241F00E
:1054000080010A4302605A68E06882F040025A60F4
:105410009A6882F040029A602946FFF7AFFF666003
:10542000628BE38A9A4206D9E3683BB19B6993F8A1
:105430002830012B02D9608BBDE8F88308A93846D3
:10544000FDF766FF0028F6D1089AD3682E44A8EB32
:105450000508258B1E60D2E901031FFA88F85968F8
:10546000454528BF454641F0800109EA05420A4307
:1054700002605A68E06882F040025A609A6882F0DE
:1054800040029A602946FFF779FFE38A2B44E382C2
:10549000C6E70020D0E700BF9408FF1F0000FF030D
:1054A0002DE9F34707460DF10600914688469A46D6
:1054B0000024FBF745FC01220178BDF80660761A4E
:1054C000B6B2ADF806604378042B15D0052B26D074
:1054D000022B07D14379BB4246D0B7FA87F464095F
:1054E000002C41D10844002EE6D1002A0CBF5046C2
:1054F000002002B0BDE8F087002CF3D0B8F1FF0F18
:1055000002D083784345EDD1B9F1FF0F02D0C378C3
:105510004B452CD1BAF1000FEBD00224E2E7002C6E
:10552000E0D0BAF1000FDDD0534616E090F802C08B
:1055300095F802E08CEA0E0C1CF07F0F0CD1022CC7
:10554000D0D095F805C02D7945EA0C25B3F804C0F4
:10555000AC45C7D29D80C5E708331D68002DE5D155
:10556000022CBFD11860BDE701240022BAE7032452
:10557000B8E737B5836993F924300546ABB1028AA1
:105580008A4212D800248DF8023001238DF80330AE
:105590000522DD23694620468DF80430ADF8004031
:1055A000FFF784FCAB6983F8244003B030BD0000F2
:1055B000F7B5114B054680781B6895F805C02A7928
:1055C000EF7800F07F062C2406FB043420F07F00E7
:1055D0000B46009442EA0C2231463843FDF7CEFEDA
:1055E000EB7823B9112384F8263003B0F0BD94F88A
:1055F000223043F00103F6E79408FF1F114B73B507
:105600001B6800F07F012C2401FB04340025E668B0
:1056100000952B462A46FF20FDF7B0FE84F8265061
:10562000658384F828501EB133683582C6E901339A
:10563000A36823B100221A821A68C3E9012202B0CA
:1056400070BD00BF9408FF1F70B58AB00C460AA950
:1056500003AB41F8203D05461646FDF759FEB0B9AB
:10566000A36993F8261041F0400183F82610606882
:10567000E168029B0093091A89B2B1420A4628BF29
:1056800032462B461146FFF799FE0AB070BD002046
:10569000FBE700002DE9F0418AB01C4680460F462A
:1056A00016469DF84050FDF735FBA31E032B00F274
:1056B000AF80DFE803F002448A3B574B1B6805EBE1
:1056C000850503EB850516F00404E9680DD08B69A8
:1056D00093F826305A0600F19B800B68CA8A4B600B
:1056E0000A824046FFF7B0FF4BE033070CD58969CB
:1056F00091F8263023F0400381F82630FDF712FBA5
:1057000020460AB0BDE8F08117F4805FAB6818BF8F
:105710000B467406996991F8263005D5D80744BF21
:1057200007F07F0481F824409CB2E7E73A4B1B68FE
:1057300005EB850503EB8505AB681C8ADEE7364B78
:105740001B6805EB850503EB8505ED68EDB90AA936
:1057500003AB41F8203D4046FDF7DAFD002857D164
:10576000B8F1000F0FD12D4B1B6863B1D9799A792D
:1057700042EA0122029B0093314643463846FFF736
:105780001DFE0446BAE73246F4E7AB6993F82640BB
:1057900014F00104B2D037B9EC8A2A8AA41AB442B0
:1057A00038DBA4B2AAE7FDF7BDFA324639462846EF
:1057B000FFF700FB0446FDF7ADFAAB6993F826301E
:1057C0005A069BD4224629468BE7134B1B6805EBF0
:1057D000850503EB85053246AD6839462846FFF757
:1057E0008CFAAB6993F826305B07044688D5FDF741
:1057F00091FAAA6992F8263023F0040382F8263041
:10580000AB6993F82500FDF755FE0028F8D075E741
:10581000002473E73C4671E77008FF1F8C08FF1FE8
:105820002DE9F041324E817B324A346805461C2313
:105830000430FFF725F995F80E800746B8F1000F00
:1058400041D02C2308FB0344AB8923836B89D90601
:1058500044BF202262845A0642BF628C42F080021A
:1058600062841B0603D5638C43F0400363841423D6
:105870006FF0130213FB07221F4B1B681344DA68F7
:10588000E26012B194612A89A282AA7B84F8252061
:105890006AB1E97B59B1608C34682C2601FB06445F
:1058A00084F8251084F82720AA89228360849B68C5
:1058B000A3601BB19C61AB7C84F824302B6823600F
:1058C0003846BDE8F081687C013000EB800300EBD6
:1058D00043008000FFF782FB08230383AB7C30602A
:1058E000044680F8243029464046FDF723FEBEE7F3
:1058F0009408FF1F955600007008FF1F2DE9F04126
:105900001646294ADDF818C012680F462C21484374
:105910001418618C09061AD5A168238B8D68D1F8FB
:105920000CE0B4F818801D4475458B8A8D6025BF46
:105930000D688D605D1C00258D82BCF1000F06D0C6
:105940008D684544AE4598BF0D68CCF80050155899
:105950001DB9A3684BB9002005E01A463146384608
:10596000A8470728F5D0BDE8F08194F9240010B1CC
:105970000421FFF76DFC638C1B06ECD494F82630F1
:1059800013F004050ED1A068C28A018A521AB242ED
:1059900004DB32463946FFF70DFADCE743F0040337
:1059A00084F826300120DEE79408FF1F2DE9F0413E
:1059B000A0B00D468022002104466846FFF789F911
:1059C0006B460022FF212846FFF76AFD60B3174EA1
:1059D0004FF000082C275DF8380010B920B0BDE862
:1059E000F08164B92DB98078FFF708FE08F101084D
:1059F000F1E70DEBC8039988FFF7DAFDF6E7827847
:105A0000336802F07F0202FB0732012C92F8263045
:105A10000BBF23F0010323F0020343F0020343F022
:105A2000010382F82630E1E70120D7E79408FF1F41
:105A30002DE9F0439446A5B00D461E4606282AD807
:105A4000DFE810F00D0178026F0207007D028B0283
:105A50009302A64B1B682C2707FB0237788BFD6847
:105A600030BBC5B12C8ADCB16A68EB689A4222BFB0
:105A7000E98A521A6A6068681B1A9AB2A24228BF61
:105A80002246009663461146FFF798FCAB6928460C
:105A9000998AFFF76EFD0024204625B0BDE8F0830B
:105AA000AA6992F8263023F0400382F82630F3E703
:105AB000FB8A984200F29A80002D78D02B8A002B26
:105AC00075D0AC6994F82810E28B012901F1FF31FF
:105AD000C9B2A3EB020388BFB4F820E084F8281011
:105AE0009BB204EB410188BFA4F81EE01E312B825B
:105AF00004F11E080022884534D1934244D1002A83
:105B000035D197F8263013F0300F15D0398BB0FB14
:105B1000F1F301FB13039BB273B9D6E901135A6881
:105B200042F088020A605A6882F040025A609A681D
:105B300082F040029A6001226B681844EB6868604A
:105B4000984224BFEB8AC01A4FF0000328BF686058
:105B50007B83002A9AD194F8263023F0400384F8FE
:105B6000263093E731F802ED724492B2C3E7628CBB
:105B700052068BD500227A83EA8A13442B82009640
:105B80006346114668687FE769680844E9686860A9
:105B9000884222BFEC8A001B68606868091A9B1A59
:105BA0008AB29342B8BF9AB200237B8369E73A8BEB
:105BB000B0FBF2F302FB13039BB2A3B9BB8B83428E
:105BC00003D197F826309B060DD5D6E901135A6804
:105BD00042F088020A605A6882F040025A609A686D
:105BE00082F040029A6000247C8355E73C8BC21A05
:105BF00093B29C4228BF1C4695B1AB6993F828200C
:105C0000D98B012A02F1FF3283F828202A8A84BF27
:105C1000188CD883521A2A82998A2846FFF7A9FC41
:105C2000F98A7B68F2680B441360D6E90103304AB5
:105C3000596802EA044241F080010A4302605A684E
:105C400082F040025A609A6882F040029A602146CF
:105C50002846FFF793FBFB8A2344FB821BE70A7865
:105C6000224B22F08004D3F800800027012CA8F8F2
:105C70001A70994600F08A80022C00F0FB80002CFC
:105C800040F03D814B78092B00F2EB80DFE813F008
:105C90007800E900E900E900E90044000A00E900B1
:105CA00072004800CB7888788F7940EA0320CB795E
:105CB00000B247EA032700F47F43B3F5007F10D01A
:105CC000B3F5407F16D0B3F5807F1BD104A8FBF756
:105CD00031F8BDF81010009600233A46FFF76EFB2E
:105CE000DAE604A8FBF72CF8F3E700BF9408FF1FDF
:105CF0000000FF0304A9C0B2FBF728F80028E8D190
:105D00000424C9E6D8F80030002BF9D0B18A00226B
:105D1000681C98470446BFE68B78B3750324BBE63E
:105D2000944E897831700020FFF740FE044610B190
:105D300000233370E4E7D9F8003093F92460002E93
:105D4000ECD0A91C01220DF11600FEF7CBFF752344
:105D50008DF8133002238DF814300722FE2304A996
:105D60002046ADF810408DF812608DF81530FFF721
:105D70009DF8D3E701220096002311467D48ADE748
:105D800002220096002311467B48A7E791F8019074
:105D9000B9F10A0F01F1020048D0B9F10B0F0CD094
:105DA000B9F1000F5DD1734B1B78002BA8D0009682
:105DB0004B4602221146714850E06E4E3378002B5C
:105DC0009ED003AA0321FFF7E4FA04AD9DF80E402C
:105DD000802239462846FEF77CFF2B46FF222146CB
:105DE0003078FFF75DFB55F83740D4B99DF80E7059
:105DF0009DF80C80802221462846FEF76AFF2B463C
:105E0000424639463078FFF74BFB00283FF478AF25
:105E100055F83400002881D00021FFF7C9FB013478
:105E2000F6E7A078FFF7EAFB0137DCE7514D2B7866
:105E3000002B3FF465AF04AA0221FFF7AAFA3B4604
:105E400022469DF810102878FFF72AFB00283FF41F
:105E500057AF00963B46224621460330FFF7AEFA85
:105E600019E6D8F80030002B3FF44AAFB18A00227F
:105E700028464EE74F78012F39D8A81C04AA21469E
:105E8000FFF787FA3B4BBDF810001B7813B90028C9
:105E90007FF436AF2C2300F01F0203FB0282012F98
:105EA00092F8261001F0080318D1002B3FF4F3AD4F
:105EB00021F0080182F82610D8F80030002B3FF4BA
:105EC000EAAD24ACC0B204F8840DFDF7F3F9D9F8BB
:105ED000003004221B68002120461AE70096002BA0
:105EE0003FF467AF0222002311462548B6E7D8F8F1
:105EF0000030002B3FF404AF03220821B8E7D8F8A4
:105F00000030002B3FF4FCAE1E4F12F0800F18BF84
:105F100039600022B18A28469847002304463B6036
:105F2000BAE5B28A32B90092022329466046FFF7E9
:105F3000E5FCEFE63369B28A00930123F5E7B37D10
:105F400033B1114B1B68CC2193F92400FEF7F2FF0B
:105F500000210846FFF72AFD9DE50B4B1B68CB216E
:105F600093F92400FEF7E6FF95E5074BCA211B686D
:105F7000F6E700BF9008FF1F9208FF1F266600008B
:105F8000246600008C08FF1F9408FF1F054B1A6849
:105F90002C2303FB002090F82630194380F82610AC
:105FA000704700BF9408FF1F034B1A682C2303FBA4
:105FB000002090F8270070479408FF1FFDF760B994
:105FC000F0B4860743D0541E002A3ED0CAB203461E
:105FD00002E014F1FF3438D303F8012B9D07F8D108
:105FE000032C2BD9CDB245EA05250F2C45EA0545F2
:105FF00016D9A4F110073F0903F1200606EB071696
:1060000003F1100242E9045542E902551032B2424E
:10601000F8D104F00F040137032C03EB07130DD95B
:106020001E462246043A032A46F8045BFAD8221F89
:1060300022F003020432134404F003042CB1C9B269
:106040001C4403F8011B9C42FBD1F0BC7047144672
:046050000346C5E757
:1060540061657332353620736563726574206B65D0
:1060640079000D0A44656C65746520636F6465206E
:106074005B792F6E5D203F203E20000D0A506C6539
:1060840061736520737461727420532D52454320EB
:10609400646F776E6C6F61643A20000D0A5374610B
:1060A4007274696E67204170706C69636174696FA2
:1060B4006E0D0A0A000D0A4D6173732065726173D7
:1060C40065205B792F6E5D203F203E20000D0A4342
:1060D4006865636B696E6720466C6173682E2E2E4B
:1060E4000020454D505459210D0A3E2000204E4FAA
:1060F4005420424C414E4B210D0A3E2000203F3F8C
:106104000D0A3E20000D0A21212044657374726F2C
:106114007920464C41534820616E64204C6F616481
:106124006572202D20636F6E6669726D205B792F16
:106134006E5D203F203E20000D0A0A44656C6574A4
:10614400696E6720636F64652E2E2E00737563631A
:1061540065737366756C0D0A3E20006661696C6533
:106164006421210D0A3E20000D0A41626F7274659C
:106174006421210D0A3E20002041626F727465641F
:10618400210D0A000D0A0A5265636F72642D65724F
:10619400726F72212120284374726C2B7220746FE9
:1061A40020726573657429000D0A0A43532D6572C4
:1061B400726F72212120284374726C2B7220746FC9
:1061C40020726573657429000D0A0A50726F677234
:1061D400616D6D696E672D6572726F722121202861
:1061E4004374726C2B7220746F207265736574290A
:1061F400000D0A0A5465726D696E61746564202D20
:106204002072657374617274696E672E2E2E00217C
:10621400000D0A0A20755461736B65722053657210
:1062240069616C204C6F61646572200056312E35B3
:10623400000D0A3D3D3D3D3D3D3D3D3D3D3D3D3D2A
:106244003D3D3D3D3D3D3D3D3D3D3D3D3D3D3D0DAA
:106254000A005B002F005D0D0A006D65203D206D76
:106264006173732065726173650D0A006263203D7A
:1062740020626C616E6B20636865636B0D0A006459
:1062840063203D2064656C65746520636F64650DEF
:106294000A006C64203D207374617274206C6F6119
:1062A400640D0A00676F203D20737461727420616D
:1062B40070706C69636174696F6E0D0A3E200069C9
:1062C4006E697469616C20766563746F720009028B
:1062D4004B000201048032080B0002020200000994
:1062E4000400000102020005052400100105240138
:1062F400010004240202052406000107058303406B
:10630400000A09040100020A000005070501024011
:106314000000070582024000000A0343006F006E7C
:1063240000660012011001EF020108A215440000EA
:1063340001010203015553422052657365740A0D2D
:10634400005553422053757370656E6465640A0D7D
:106354000055534220526573756D650A0D00456EF4
:10636400756D6572617465640D0A00080349006EF9
:106374000074000A034D0061006E00750010034DA7
:106384000079002000500072006F0064000A03309E
:106394000030003000310000B46300007763000077
:1063A40081630000916300001D6300006F630000BF
:1063B4000403090473645F636172645F616573322B
:1063C40035365F636F6465642E62696E00A748B6F4
:1063D4005311244E6F6E2D666F726D617474656413
:1063E400200053442D636172640D0A0053442D63ED
:1063F400617264206E6F7420726573706F6E64696D
:106404006E670D0A0053442D6361726420766F6CCD
:1064140074616765206572726F720D0A0053442DB2
:1064240063617264205631206F72204D4D43202DDC
:10643400206E6F7420737570706F72746564210DB3
:106444000A0053442D63617264205632202D2000CB
:10645400486967682043617061636974790D0A0053
:106464007374616E646172640D0A004D616C666FD1
:10647400726D6564202D20004E4F542046415431E6
:10648400362D20004469736B2044206D6F756E7443
:10649400656400443A5C0000010000000000000054
:1064A4000101000000021010101010101010101044
:1064B40001010101010000040404040404040404AF
:1064C4000404040404040404040404040404040488
:1064D400042002200000000808080808080808082A
:1064E4000808080808080808080808080808080828
:1064F400080020000000000000009508000001AA28
:106504008702000000002940FF8000100002000202
:106514000300000000203120353032203530322095
:10652400004A616E00466562004D617200417072FE
:10653400004D6179004A756E004A756C00417567BB
:1065440000536570004F6374004E6F7600446563BA
:1065540000203C4449523E2020202020202020209E
:10656400202000015748754D53610000010000C010
:1065740000000000E5650000BD5F000000000000B1
:1065840002000100EA6500007D08000045000200E9
:1065940000000000EE650000190C00002500FFFF5C
:1065A40000000400F2650000291A00004500FFFF06
:1065B40000000400F9650000151000002500FFFF2D
:1065C40000000400000000000000000000000000C3
:1065D4000000000054494D454F55542121210D0A16
:1065E4000057646F670061707000757362004D61DD
:1065F400737353740053440000E1F50580969800CA
:1066040040420F00A086010010270000E8030000AC
:10661400640000000A000000010000000000000007
:046624000100000071
:106628003700000000070000000009000000000615
:106638000000000201008021017001780906FCD5E4
:10664800704700000000000000000000000000008B
:106658007002FF1F000040A8001008E000000000C2
:10666800A41A95A8000057A9081B08E0881808E094
:10667800481808E0001008E00000000000000000D2
:10668800B4AA15BC0090D5AC481B08E0881808E0EF
:10669800481808E0001008E00000000000000000B2
:1066A80000000001000000020000000400000008D3
:1066B80000000010000000200000004000000080E2
:0966C8000000001B00000036FF79
:0400000300000410E5
:00000001FF
